 popframe009

 Timestamp is 9d7d36e4 (reproducible build file hash)

 Preferred load address is 0000000180000000

 Start         Length     Name                   Class
 0001:00000000 00003a30H .text$mn                CODE
 0001:00003a30 00000036H .text$mn$00             CODE
 0001:00003a66 00000092H .text$x                 CODE
 0002:00000000 00000198H .idata$5                DATA
 0002:00000198 00000038H .00cfg                  DATA
 0002:000001d0 00000008H .CRT$XCA                DATA
 0002:000001d8 00000008H .CRT$XCZ                DATA
 0002:000001e0 00000008H .CRT$XIA                DATA
 0002:000001e8 00000008H .CRT$XIC                DATA
 0002:000001f0 00000008H .CRT$XIZ                DATA
 0002:000001f8 00000008H .CRT$XLA                DATA
 0002:00000200 00000008H .CRT$XLZ                DATA
 0002:00000208 00000008H .CRT$XPA                DATA
 0002:00000210 00000008H .CRT$XPZ                DATA
 0002:00000218 00000008H .CRT$XTA                DATA
 0002:00000220 00000010H .CRT$XTZ                DATA
 0002:00000228 00000000H .gehcont$y              DATA
 0002:00000228 00000000H .gfids$y                DATA
 0002:00000230 00002250H .rdata                  DATA
 0002:00002480 00000000H .rdata$CastGuardVftablesA DATA
 0002:00002480 00000000H .rdata$CastGuardVftablesC DATA
 0002:00002480 00000028H .rdata$T                DATA
 0002:000024a8 000000a4H .rdata$voltmd           DATA
 0002:0000254c 0000031cH .rdata$zzzdbg           DATA
 0002:00002868 00000008H .rtc$IAA                DATA
 0002:00002870 00000008H .rtc$IZZ                DATA
 0002:00002878 00000008H .rtc$TAA                DATA
 0002:00002880 00000008H .rtc$TZZ                DATA
 0002:00002888 00000004H .tls                    DATA
 0002:0000288c 00000004H .tls$                   DATA
 0002:00002890 00000008H .tls$ZZZ                DATA
 0002:00002898 00000308H .xdata                  DATA
 0002:00002ba0 000003d0H .edata                  DATA
 0002:00002f70 00000064H .idata$2                DATA
 0002:00002fd4 00000014H .idata$3                DATA
 0002:00002fe8 00000198H .idata$4                DATA
 0002:00003180 0000041eH .idata$6                DATA
 0003:00000000 00000080H .data                   DATA
 0003:00000080 0001b3a8H .bss                    DATA
 0004:00000000 000003a8H .pdata                  DATA

  Address         Publics by Value              Rva+Base               Lib:Object

 0000:00000000       __AbsoluteZero             0000000000000000     <absolute>
 0000:00000000       ___safe_se_handler_count   0000000000000000     <absolute>
 0000:00000000       ___safe_se_handler_table   0000000000000000     <absolute>
 0000:00000000       __arm64x_extra_rfe_table   0000000000000000     <absolute>
 0000:00000000       __arm64x_extra_rfe_table_size 0000000000000000     <absolute>
 0000:00000000       __arm64x_native_entrypoint 0000000000000000     <absolute>
 0000:00000000       __arm64x_redirection_metadata 0000000000000000     <absolute>
 0000:00000000       __arm64x_redirection_metadata_count 0000000000000000     <absolute>
 0000:00000000       __dynamic_value_reloc_table 0000000000000000     <absolute>
 0000:00000000       __enclave_config           0000000000000000     <absolute>
 0000:00000000       __guard_check_icall_a64n_fptr 0000000000000000     <absolute>
 0000:00000000       __guard_eh_cont_count      0000000000000000     <absolute>
 0000:00000000       __guard_eh_cont_table      0000000000000000     <absolute>
 0000:00000000       __guard_fids_count         0000000000000000     <absolute>
 0000:00000000       __guard_fids_table         0000000000000000     <absolute>
 0000:00000000       __guard_iat_count          0000000000000000     <absolute>
 0000:00000000       __guard_iat_table          0000000000000000     <absolute>
 0000:00000000       __guard_longjmp_count      0000000000000000     <absolute>
 0000:00000000       __guard_longjmp_table      0000000000000000     <absolute>
 0000:00000000       __hybrid_auxiliary_iat     0000000000000000     <absolute>
 0000:00000000       __hybrid_auxiliary_iat_copy 0000000000000000     <absolute>
 0000:00000000       __hybrid_code_map          0000000000000000     <absolute>
 0000:00000000       __hybrid_code_map_count    0000000000000000     <absolute>
 0000:00000000       __x64_code_ranges_to_entry_points 0000000000000000     <absolute>
 0000:00000000       __x64_code_ranges_to_entry_points_count 0000000000000000     <absolute>
 0000:00000100       __guard_flags              0000000000000100     <absolute>
 0000:00000000       __ImageBase                0000000180000000     <linker-defined>
 0001:00000000       ?NewObject@JNIEnv_@@QEAAPEAV_jobject@@PEAV_jclass@@PEAU_jmethodID@@ZZ 0000000180001000 f i libpopframe009.obj
 0001:00000028       ?SetEventNotificationMode@_jvmtiEnv@@QEAA?AW4jvmtiError@@W4jvmtiEventMode@@W4jvmtiEvent@@PEAV_jobject@@ZZ 0000000180001028 f i libpopframe009.obj
 0001:00000034       ?TranslateError@@YAPEBDW4jvmtiError@@@Z 0000000180001034 f   libpopframe009.obj
 0001:000002ec       ?nsk_jni_check_exception@@YAHPEAUJNIEnv_@@QEBDH@Z 00000001800012ec f   libpopframe009.obj
 0001:00000430       ?nsk_jni_lverify@@YAHHPEAUJNIEnv_@@HQEBDH1ZZ 0000000180001430 f   libpopframe009.obj
 0001:000004d0       Agent_Initialize           00000001800014d0 f   libpopframe009.obj
 0001:0000069c       Agent_OnAttach             000000018000169c f   libpopframe009.obj
 0001:0000069c       Agent_OnLoad               000000018000169c f   libpopframe009.obj
 0001:000006a4       Breakpoint                 00000001800016a4 f   libpopframe009.obj
 0001:00000808       Java_nsk_jvmti_PopFrame_popframe009_check 0000000180001808 f   libpopframe009.obj
 0001:000010cc       Java_nsk_jvmti_PopFrame_popframe009_getReady 00000001800020cc f   libpopframe009.obj
 0001:00001200       Java_nsk_jvmti_unit_FollowReferences_FollowRefObjects_addRefToVerify 0000000180002200 f   libpopframe009.obj
 0001:000013d8       Java_nsk_jvmti_unit_FollowReferences_FollowRefObjects_getTag 00000001800023d8 f   libpopframe009.obj
 0001:00001498       Java_nsk_jvmti_unit_FollowReferences_FollowRefObjects_resetRefsToVerify 0000000180002498 f   libpopframe009.obj
 0001:000014a0       Java_nsk_jvmti_unit_FollowReferences_FollowRefObjects_resetTags 00000001800024a0 f   libpopframe009.obj
 0001:000014e4       Java_nsk_jvmti_unit_FollowReferences_FollowRefObjects_setTag 00000001800024e4 f   libpopframe009.obj
 0001:0000173c       Java_nsk_share_jvmti_ArgumentHandler_getAgentOptionsString 000000018000273c f   libpopframe009.obj
 0001:000017ec       Java_nsk_share_jvmti_DebugeeClass_checkStatus 00000001800027ec f   libpopframe009.obj
 0001:00001874       Java_nsk_share_jvmti_DebugeeClass_resetAgentData 0000000180002874 f   libpopframe009.obj
 0001:000018d4       Java_nsk_share_jvmti_RedefineAgent_agentStatus 00000001800028d4 f   libpopframe009.obj
 0001:000018e0       Java_nsk_share_jvmti_RedefineAgent_isRedefined 00000001800028e0 f   libpopframe009.obj
 0001:000018ec       Java_nsk_share_jvmti_RedefineAgent_redefineAttempted 00000001800028ec f   libpopframe009.obj
 0001:000018f8       MA_checkStatus             00000001800028f8 f   libpopframe009.obj
 0001:0000199c       SingleStep                 000000018000299c f   libpopframe009.obj
 0001:00001b64       __local_stdio_printf_options 0000000180002b64 f i libpopframe009.obj
 0001:00001d44       exitOnError                0000000180002d44 f   libpopframe009.obj
 0001:00001df8       fprintf                    0000000180002df8 f i libpopframe009.obj
 0001:00001e3c       nsk_jvmti_lverify          0000000180002e3c f   libpopframe009.obj
 0001:00001f2c       nsk_jvmti_resetAgentData   0000000180002f2c f   libpopframe009.obj
 0001:00001fac       nsk_jvmti_setFailStatus    0000000180002fac f   libpopframe009.obj
 0001:00001fe8       nsk_lcomplain              0000000180002fe8 f   libpopframe009.obj
 0001:00002008       nsk_ldisplay               0000000180003008 f   libpopframe009.obj
 0001:00002028       nsk_ltrace                 0000000180003028 f   libpopframe009.obj
 0001:00002048       nsk_lvcomplain             0000000180003048 f   libpopframe009.obj
 0001:00002200       nsk_lvdisplay              0000000180003200 f   libpopframe009.obj
 0001:0000224c       nsk_lverify                000000018000324c f   libpopframe009.obj
 0001:000022a8       nsk_lvtrace                00000001800032a8 f   libpopframe009.obj
 0001:00002308       nsk_printf                 0000000180003308 f   libpopframe009.obj
 0001:00002330       nsk_vprintf                0000000180003330 f   libpopframe009.obj
 0001:000023e4       popFrames                  00000001800033e4 f   libpopframe009.obj
 0001:000025e0       printf                     00000001800035e0 f i libpopframe009.obj
 0001:00002b08       __raise_securityfailure    0000000180003b08 f   MSVCRT:gs_report.obj
 0001:00002b3c       __report_gsfailure         0000000180003b3c f   MSVCRT:gs_report.obj
 0001:00002d7c       __GSHandlerCheck           0000000180003d7c f   MSVCRT:gshandler.obj
 0001:00002d9c       __GSHandlerCheckCommon     0000000180003d9c f   MSVCRT:gshandler.obj
 0001:00002e10       __security_check_cookie    0000000180003e10 f   MSVCRT:amdsecgs.obj
 0001:00003150       _DllMainCRTStartup         0000000180004150 f   MSVCRT:dll_dllmain.obj
 0001:00003190       __scrt_acquire_startup_lock 0000000180004190 f   MSVCRT:utility.obj
 0001:000031cc       __scrt_dllmain_after_initialize_c 00000001800041cc f   MSVCRT:utility.obj
 0001:00003200       __scrt_dllmain_before_initialize_c 0000000180004200 f   MSVCRT:utility.obj
 0001:00003218       __scrt_dllmain_crt_thread_attach 0000000180004218 f   MSVCRT:utility.obj
 0001:00003240       __scrt_dllmain_crt_thread_detach 0000000180004240 f   MSVCRT:utility.obj
 0001:00003258       __scrt_dllmain_exception_filter 0000000180004258 f   MSVCRT:utility.obj
 0001:000032b8       __scrt_dllmain_uninitialize_c 00000001800042b8 f   MSVCRT:utility.obj
 0001:000032e8       __scrt_dllmain_uninitialize_critical 00000001800042e8 f   MSVCRT:utility.obj
 0001:000032fc       __scrt_initialize_crt      00000001800042fc f   MSVCRT:utility.obj
 0001:00003348       __scrt_initialize_onexit_tables 0000000180004348 f   MSVCRT:utility.obj
 0001:000033d4       __scrt_is_nonwritable_in_current_image 00000001800043d4 f   MSVCRT:utility.obj
 0001:0000346c       __scrt_release_startup_lock 000000018000446c f   MSVCRT:utility.obj
 0001:00003490       __scrt_uninitialize_crt    0000000180004490 f   MSVCRT:utility.obj
 0001:000034bc       _onexit                    00000001800044bc f   MSVCRT:utility.obj
 0001:000034f8       atexit                     00000001800044f8 f   MSVCRT:utility.obj
 0001:00003510       __crt_debugger_hook        0000000180004510 f   MSVCRT:utility_desktop.obj
 0001:00003518       __scrt_fastfail            0000000180004518 f   MSVCRT:utility_desktop.obj
 0001:00003664       _guard_check_icall_nop     0000000180004664 f i MSVCRT:guard_support.obj
 0001:00003668       __security_init_cookie     0000000180004668 f   MSVCRT:gs_support.obj
 0001:00003714       DllMain                    0000000180004714 f   MSVCRT:dll_dllmain_stub.obj
 0001:00003738       ?__scrt_initialize_type_info@@YAXXZ 0000000180004738 f   MSVCRT:tncleanup.obj
 0001:00003748       ?__scrt_uninitialize_type_info@@YAXXZ 0000000180004748 f   MSVCRT:tncleanup.obj
 0001:00003754       __local_stdio_scanf_options 0000000180004754 f i MSVCRT:default_local_stdio_options.obj
 0001:0000375c       __scrt_initialize_default_local_stdio_options 000000018000475c f   MSVCRT:default_local_stdio_options.obj
 0001:00003778       __scrt_get_dyn_tls_init_callback 0000000180004778 f   MSVCRT:dyn_tls_init.obj
 0001:00003780       _RTC_Initialize            0000000180004780 f   MSVCRT:initsect.obj
 0001:000037bc       _RTC_Terminate             00000001800047bc f   MSVCRT:initsect.obj
 0001:000037f8       __isa_available_init       00000001800047f8 f   MSVCRT:cpu_disp.obj
 0001:000039a4       _get_startup_argv_mode     00000001800049a4 f   MSVCRT:argv_mode.obj
 0001:000039ac       __scrt_is_ucrt_dll_in_use  00000001800049ac f   MSVCRT:ucrt_detection.obj
 0001:000039c0       memcpy                     00000001800049c0 f   vcruntime:VCRUNTIME140.dll
 0001:000039c6       memset                     00000001800049c6 f   vcruntime:VCRUNTIME140.dll
 0001:000039cc       strchr                     00000001800049cc f   vcruntime:VCRUNTIME140.dll
 0001:000039d2       __C_specific_handler       00000001800049d2 f   vcruntime:VCRUNTIME140.dll
 0001:000039d8       __std_type_info_destroy_list 00000001800049d8 f   vcruntime:VCRUNTIME140.dll
 0001:000039de       strcmp                     00000001800049de f   ucrt:api-ms-win-crt-string-l1-1-0.dll
 0001:000039e4       strlen                     00000001800049e4 f   ucrt:api-ms-win-crt-string-l1-1-0.dll
 0001:000039ea       _initterm                  00000001800049ea f   ucrt:api-ms-win-crt-runtime-l1-1-0.dll
 0001:000039f0       _initterm_e                00000001800049f0 f   ucrt:api-ms-win-crt-runtime-l1-1-0.dll
 0001:000039f6       _seh_filter_dll            00000001800049f6 f   ucrt:api-ms-win-crt-runtime-l1-1-0.dll
 0001:000039fc       _configure_narrow_argv     00000001800049fc f   ucrt:api-ms-win-crt-runtime-l1-1-0.dll
 0001:00003a02       _initialize_narrow_environment 0000000180004a02 f   ucrt:api-ms-win-crt-runtime-l1-1-0.dll
 0001:00003a08       _initialize_onexit_table   0000000180004a08 f   ucrt:api-ms-win-crt-runtime-l1-1-0.dll
 0001:00003a0e       _register_onexit_function  0000000180004a0e f   ucrt:api-ms-win-crt-runtime-l1-1-0.dll
 0001:00003a14       _execute_onexit_table      0000000180004a14 f   ucrt:api-ms-win-crt-runtime-l1-1-0.dll
 0001:00003a1a       _crt_atexit                0000000180004a1a f   ucrt:api-ms-win-crt-runtime-l1-1-0.dll
 0001:00003a20       _cexit                     0000000180004a20 f   ucrt:api-ms-win-crt-runtime-l1-1-0.dll
 0001:00003a28       __acrt_initialize          0000000180004a28 f   MSVCRT:ucrt_stubs.obj
 0001:00003a28       __acrt_thread_attach       0000000180004a28 f   MSVCRT:ucrt_stubs.obj
 0001:00003a28       __acrt_thread_detach       0000000180004a28 f   MSVCRT:ucrt_stubs.obj
 0001:00003a28       __acrt_uninitialize        0000000180004a28 f   MSVCRT:ucrt_stubs.obj
 0001:00003a28       __acrt_uninitialize_critical 0000000180004a28 f   MSVCRT:ucrt_stubs.obj
 0001:00003a28       __scrt_stub_for_acrt_initialize 0000000180004a28 f   MSVCRT:ucrt_stubs.obj
 0001:00003a28       __scrt_stub_for_acrt_thread_attach 0000000180004a28 f   MSVCRT:ucrt_stubs.obj
 0001:00003a28       __scrt_stub_for_acrt_thread_detach 0000000180004a28 f   MSVCRT:ucrt_stubs.obj
 0001:00003a28       __scrt_stub_for_acrt_uninitialize 0000000180004a28 f   MSVCRT:ucrt_stubs.obj
 0001:00003a28       __scrt_stub_for_acrt_uninitialize_critical 0000000180004a28 f   MSVCRT:ucrt_stubs.obj
 0001:00003a28       __vcrt_initialize          0000000180004a28 f   MSVCRT:ucrt_stubs.obj
 0001:00003a28       __vcrt_thread_attach       0000000180004a28 f   MSVCRT:ucrt_stubs.obj
 0001:00003a28       __vcrt_thread_detach       0000000180004a28 f   MSVCRT:ucrt_stubs.obj
 0001:00003a28       __vcrt_uninitialize        0000000180004a28 f   MSVCRT:ucrt_stubs.obj
 0001:00003a28       __vcrt_uninitialize_critical 0000000180004a28 f   MSVCRT:ucrt_stubs.obj
 0001:00003a2c       __scrt_stub_for_is_c_termination_complete 0000000180004a2c f   MSVCRT:ucrt_stubs.obj
 0001:00003a2c       _is_c_termination_complete 0000000180004a2c f   MSVCRT:ucrt_stubs.obj
 0001:00003a40       _guard_dispatch_icall_nop  0000000180004a40 f   MSVCRT:guard_dispatch.obj
 0001:00003a60       _guard_xfg_dispatch_icall_nop 0000000180004a60 f   MSVCRT:guard_xfg_dispatch.obj
 0002:00000000       __imp_RtlCaptureContext    0000000180005000     kernel32:KERNEL32.dll
 0002:00000008       __imp_RtlLookupFunctionEntry 0000000180005008     kernel32:KERNEL32.dll
 0002:00000010       __imp_RtlVirtualUnwind     0000000180005010     kernel32:KERNEL32.dll
 0002:00000018       __imp_UnhandledExceptionFilter 0000000180005018     kernel32:KERNEL32.dll
 0002:00000020       __imp_SetUnhandledExceptionFilter 0000000180005020     kernel32:KERNEL32.dll
 0002:00000028       __imp_GetCurrentProcess    0000000180005028     kernel32:KERNEL32.dll
 0002:00000030       __imp_TerminateProcess     0000000180005030     kernel32:KERNEL32.dll
 0002:00000038       __imp_IsProcessorFeaturePresent 0000000180005038     kernel32:KERNEL32.dll
 0002:00000040       __imp_CloseHandle          0000000180005040     kernel32:KERNEL32.dll
 0002:00000048       __imp_InitializeCriticalSectionAndSpinCount 0000000180005048     kernel32:KERNEL32.dll
 0002:00000050       __imp_DeleteCriticalSection 0000000180005050     kernel32:KERNEL32.dll
 0002:00000058       __imp_CreateEventW         0000000180005058     kernel32:KERNEL32.dll
 0002:00000060       __imp_GetModuleHandleW     0000000180005060     kernel32:KERNEL32.dll
 0002:00000068       __imp_GetProcAddress       0000000180005068     kernel32:KERNEL32.dll
 0002:00000070       __imp_IsDebuggerPresent    0000000180005070     kernel32:KERNEL32.dll
 0002:00000078       __imp_QueryPerformanceCounter 0000000180005078     kernel32:KERNEL32.dll
 0002:00000080       __imp_GetCurrentProcessId  0000000180005080     kernel32:KERNEL32.dll
 0002:00000088       __imp_GetCurrentThreadId   0000000180005088     kernel32:KERNEL32.dll
 0002:00000090       __imp_GetSystemTimeAsFileTime 0000000180005090     kernel32:KERNEL32.dll
 0002:00000098       __imp_DisableThreadLibraryCalls 0000000180005098     kernel32:KERNEL32.dll
 0002:000000a0       __imp_InitializeSListHead  00000001800050a0     kernel32:KERNEL32.dll
 0002:000000a8       \177KERNEL32_NULL_THUNK_DATA 00000001800050a8     kernel32:KERNEL32.dll
 0002:000000b0       __imp_memcpy               00000001800050b0     vcruntime:VCRUNTIME140.dll
 0002:000000b8       __imp_memset               00000001800050b8     vcruntime:VCRUNTIME140.dll
 0002:000000c0       __imp_strchr               00000001800050c0     vcruntime:VCRUNTIME140.dll
 0002:000000c8       __imp___C_specific_handler 00000001800050c8     vcruntime:VCRUNTIME140.dll
 0002:000000d0       __imp___std_type_info_destroy_list 00000001800050d0     vcruntime:VCRUNTIME140.dll
 0002:000000d8       \177VCRUNTIME140_NULL_THUNK_DATA 00000001800050d8     vcruntime:VCRUNTIME140.dll
 0002:000000e0       __imp__errno               00000001800050e0     ucrt:api-ms-win-crt-runtime-l1-1-0.dll
 0002:000000e8       __imp_exit                 00000001800050e8     ucrt:api-ms-win-crt-runtime-l1-1-0.dll
 0002:000000f0       __imp__cexit               00000001800050f0     ucrt:api-ms-win-crt-runtime-l1-1-0.dll
 0002:000000f8       __imp__crt_atexit          00000001800050f8     ucrt:api-ms-win-crt-runtime-l1-1-0.dll
 0002:00000100       __imp__execute_onexit_table 0000000180005100     ucrt:api-ms-win-crt-runtime-l1-1-0.dll
 0002:00000108       __imp__register_onexit_function 0000000180005108     ucrt:api-ms-win-crt-runtime-l1-1-0.dll
 0002:00000110       __imp__initialize_onexit_table 0000000180005110     ucrt:api-ms-win-crt-runtime-l1-1-0.dll
 0002:00000118       __imp__initialize_narrow_environment 0000000180005118     ucrt:api-ms-win-crt-runtime-l1-1-0.dll
 0002:00000120       __imp__configure_narrow_argv 0000000180005120     ucrt:api-ms-win-crt-runtime-l1-1-0.dll
 0002:00000128       __imp__seh_filter_dll      0000000180005128     ucrt:api-ms-win-crt-runtime-l1-1-0.dll
 0002:00000130       __imp__initterm_e          0000000180005130     ucrt:api-ms-win-crt-runtime-l1-1-0.dll
 0002:00000138       __imp__initterm            0000000180005138     ucrt:api-ms-win-crt-runtime-l1-1-0.dll
 0002:00000140       \177api-ms-win-crt-runtime-l1-1-0_NULL_THUNK_DATA 0000000180005140     ucrt:api-ms-win-crt-runtime-l1-1-0.dll
 0002:00000148       __imp___acrt_iob_func      0000000180005148     ucrt:api-ms-win-crt-stdio-l1-1-0.dll
 0002:00000150       __imp_fflush               0000000180005150     ucrt:api-ms-win-crt-stdio-l1-1-0.dll
 0002:00000158       __imp___stdio_common_vsprintf 0000000180005158     ucrt:api-ms-win-crt-stdio-l1-1-0.dll
 0002:00000160       __imp___stdio_common_vfprintf 0000000180005160     ucrt:api-ms-win-crt-stdio-l1-1-0.dll
 0002:00000168       \177api-ms-win-crt-stdio-l1-1-0_NULL_THUNK_DATA 0000000180005168     ucrt:api-ms-win-crt-stdio-l1-1-0.dll
 0002:00000170       __imp_strcmp               0000000180005170     ucrt:api-ms-win-crt-string-l1-1-0.dll
 0002:00000178       __imp__strdup              0000000180005178     ucrt:api-ms-win-crt-string-l1-1-0.dll
 0002:00000178       __imp_strdup               0000000180005178     ucrt:api-ms-win-crt-string-l1-1-0.dll
 0002:00000180       __imp_strlen               0000000180005180     ucrt:api-ms-win-crt-string-l1-1-0.dll
 0002:00000188       __imp_strncpy              0000000180005188     ucrt:api-ms-win-crt-string-l1-1-0.dll
 0002:00000190       \177api-ms-win-crt-string-l1-1-0_NULL_THUNK_DATA 0000000180005190     ucrt:api-ms-win-crt-string-l1-1-0.dll
 0002:00000198       __guard_check_icall_fptr   0000000180005198     MSVCRT:guard_support.obj
 0002:000001a0       __guard_xfg_check_icall_fptr 00000001800051a0     MSVCRT:guard_support.obj
 0002:000001a8       __guard_dispatch_icall_fptr 00000001800051a8     MSVCRT:guard_support.obj
 0002:000001b0       __guard_xfg_dispatch_icall_fptr 00000001800051b0     MSVCRT:guard_support.obj
 0002:000001b8       __guard_xfg_table_dispatch_icall_fptr 00000001800051b8     MSVCRT:guard_support.obj
 0002:000001c0       __castguard_check_failure_os_handled_fptr 00000001800051c0     MSVCRT:guard_support.obj
 0002:000001c8       __guard_memcpy_fptr        00000001800051c8     vcruntime:softmemtag.obj
 0002:000001d0       __xc_a                     00000001800051d0     MSVCRT:initializers.obj
 0002:000001d8       __xc_z                     00000001800051d8     MSVCRT:initializers.obj
 0002:000001e0       __xi_a                     00000001800051e0     MSVCRT:initializers.obj
 0002:000001f0       __xi_z                     00000001800051f0     MSVCRT:initializers.obj
 0002:000001f8       __xl_a                     00000001800051f8     MSVCRT:tlssup.obj
 0002:00000200       __xl_z                     0000000180005200     MSVCRT:tlssup.obj
 0002:00000208       __xp_a                     0000000180005208     MSVCRT:initializers.obj
 0002:00000210       __xp_z                     0000000180005210     MSVCRT:initializers.obj
 0002:00000218       __xt_a                     0000000180005218     MSVCRT:initializers.obj
 0002:00000220       __xt_z                     0000000180005220     MSVCRT:initializers.obj
 0002:00000230       g_refKindStr               0000000180005230     libpopframe009.obj
 0002:000003e0       ??_C@_09BPLDFGCI@unknown_0@ 00000001800053e0     libpopframe009.obj
 0002:000003f0       ??_C@_0BL@FPNMECJD@JVMTI_HEAP_REFERENCE_CLASS@ 00000001800053f0     libpopframe009.obj
 0002:00000410       ??_C@_0BL@FKGKKLNM@JVMTI_HEAP_REFERENCE_FIELD@ 0000000180005410     libpopframe009.obj
 0002:00000430       ??_C@_0CD@CAEHCFJF@JVMTI_HEAP_REFERENCE_ARRAY_ELEM@ 0000000180005430     libpopframe009.obj
 0002:00000458       ??_C@_0CC@DNEBMCNK@JVMTI_HEAP_REFERENCE_CLASS_LOAD@ 0000000180005458     libpopframe009.obj
 0002:00000480       ??_C@_0BN@CJMIPEBB@JVMTI_HEAP_REFERENCE_SIGNERS@ 0000000180005480     libpopframe009.obj
 0002:000004a0       ??_C@_0CH@HBOIDPEB@JVMTI_HEAP_REFERENCE_PROTECTION@ 00000001800054a0     libpopframe009.obj
 0002:000004c8       ??_C@_0BP@MDKGDGKL@JVMTI_HEAP_REFERENCE_INTERFACE@ 00000001800054c8     libpopframe009.obj
 0002:000004e8       ??_C@_0CC@JJMIHNJH@JVMTI_HEAP_REFERENCE_STATIC_FIE@ 00000001800054e8     libpopframe009.obj
 0002:00000510       ??_C@_0CD@IDHEEGID@JVMTI_HEAP_REFERENCE_CONSTANT_P@ 0000000180005510     libpopframe009.obj
 0002:00000538       ??_C@_0CA@EFFCHNG@JVMTI_HEAP_REFERENCE_SUPERCLASS@ 0000000180005538     libpopframe009.obj
 0002:00000558       ??_C@_0L@PCDFHGCJ@unknown_11@ 0000000180005558     libpopframe009.obj
 0002:00000568       ??_C@_0L@NJBICFOK@unknown_12@ 0000000180005568     libpopframe009.obj
 0002:00000578       ??_C@_0L@MAADBEKL@unknown_13@ 0000000180005578     libpopframe009.obj
 0002:00000588       ??_C@_0L@IPECICGM@unknown_14@ 0000000180005588     libpopframe009.obj
 0002:00000598       ??_C@_0L@JGFJLDCN@unknown_15@ 0000000180005598     libpopframe009.obj
 0002:000005a8       ??_C@_0L@LNHEOAOO@unknown_16@ 00000001800055a8     libpopframe009.obj
 0002:000005b8       ??_C@_0L@KEGPNBKP@unknown_17@ 00000001800055b8     libpopframe009.obj
 0002:000005c8       ??_C@_0L@CDPHMNGA@unknown_18@ 00000001800055c8     libpopframe009.obj
 0002:000005d8       ??_C@_0L@DKOMPMCB@unknown_19@ 00000001800055d8     libpopframe009.obj
 0002:000005e8       ??_C@_0L@OJGIPJDB@unknown_20@ 00000001800055e8     libpopframe009.obj
 0002:000005f8       ??_C@_0CA@KAOFNDEM@JVMTI_HEAP_REFERENCE_JNI_GLOBAL@ 00000001800055f8     libpopframe009.obj
 0002:00000618       ??_C@_0CC@HPFAJBK@JVMTI_HEAP_REFERENCE_SYSTEM_CLA@ 0000000180005618     libpopframe009.obj
 0002:00000640       ??_C@_0BN@FDEGFOHC@JVMTI_HEAP_REFERENCE_MONITOR@ 0000000180005640     libpopframe009.obj
 0002:00000660       ??_C@_0CB@HKIBCMAJ@JVMTI_HEAP_REFERENCE_STACK_LOCA@ 0000000180005660     libpopframe009.obj
 0002:00000688       ??_C@_0BP@EAACMMOE@JVMTI_HEAP_REFERENCE_JNI_LOCAL@ 0000000180005688     libpopframe009.obj
 0002:000006a8       ??_C@_0BM@IJDEOGOE@JVMTI_HEAP_REFERENCE_THREAD@ 00000001800056a8     libpopframe009.obj
 0002:000006c8       ??_C@_0BL@EDGPPKC@JVMTI_HEAP_REFERENCE_OTHER@ 00000001800056c8     libpopframe009.obj
 0002:000006e4       ??_C@_04BCJPDBDA@Code@     00000001800056e4     libpopframe009.obj
 0002:000006f0       ??_C@_0BA@OCLMCFKC@LineNumberTable@ 00000001800056f0     libpopframe009.obj
 0002:00000700       ??_C@_0BD@CPAEPILC@LocalVariableTable@ 0000000180005700     libpopframe009.obj
 0002:00000718       ??_C@_0BH@NMBDNHBD@LocalVariableTypeTable@ 0000000180005718     libpopframe009.obj
 0002:00000730       ??_C@_0O@HIHEEDNJ@StackMapTable@ 0000000180005730     libpopframe009.obj
 0002:00000740       ??_C@_0L@HCDIAMJG@?9?5?$CFs?0?5?$CFd?3?5@ 0000000180005740     libpopframe009.obj
 0002:00000750       ??_C@_0JI@HLPECLFI@?$CD?5?4?4?4?6?$CD?5ERROR?3?5too?5many?5complai@ 0000000180005750     libpopframe009.obj
 0002:000007f0       ??_C@_0ED@JNEKCCOB@The?5following?5fake?5exception?5st@ 00000001800057f0     libpopframe009.obj
 0002:00000838       ??_C@_0CN@FCNMDFBH@nsk?4share?4Fake_Exception_for_RU@ 0000000180005838     libpopframe009.obj
 0002:00000868       ??_C@_08PGFFNAEI@?$CI?$CFs?3?$CFd?$CJ?5@ 0000000180005868     libpopframe009.obj
 0002:00000878       ??_C@_0DP@IENMAEGI@s?2test?2hotspot?2jtreg?2vmTestbase@ 0000000180005878     libpopframe009.obj
 0002:000008b8       ??_C@_0BL@NDJLFFJB@?7at?5nsk_lvcomplain?$CI?$CFs?3?$CFd?$CJ?6@ 00000001800058b8     libpopframe009.obj
 0002:000008d8       ??_C@_0BC@JOOKAFKF@?$CD?5ERROR?3?5?$CFs?0?5?$CFd?3?5@ 00000001800058d8     libpopframe009.obj
 0002:000008f0       ??_C@_09KJEAHMEH@?$CD?5ERROR?3?5@ 00000001800058f0     libpopframe009.obj
 0002:000008fc       ??_C@_02GPIOPFAK@?$DO?$DO@ 00000001800058fc     libpopframe009.obj
 0002:00000900       ??_C@_02FODMEDOG@?$DM?$DM@ 0000000180005900     libpopframe009.obj
 0002:00000904       ??_C@_02DJGKEECL@?4?4@     0000000180005904     libpopframe009.obj
 0002:00000908       ??_C@_0O@CJPGJOAF@?9?5?$CFs?0?5?$CFd?3?5?$CFs?5@ 0000000180005908     libpopframe009.obj
 0002:00000918       ??_C@_0CB@IAKPDOIC@?$CD?5?5?5verified?5assertion?5is?5FALSE@ 0000000180005918     libpopframe009.obj
 0002:00000940       ??_C@_0CO@LGONDEPD@stdout?3?5fflush?5failed?5?9?5err?$DN?$CFd?5@ 0000000180005940     libpopframe009.obj
 0002:00000970       ??_C@_0CO@KBGKJPBD@stderr?3?5fflush?5failed?5?9?5err?$DN?$CFd?5@ 0000000180005970     libpopframe009.obj
 0002:000009a0       ??_C@_0BB@JCNMKLLK@JVMTI_ERROR_NONE@ 00000001800059a0     libpopframe009.obj
 0002:000009b8       ??_C@_0BL@LDIMKLPH@JVMTI_ERROR_INVALID_THREAD@ 00000001800059b8     libpopframe009.obj
 0002:000009d8       ??_C@_0CB@PJFPAIKJ@JVMTI_ERROR_INVALID_THREAD_GROU@ 00000001800059d8     libpopframe009.obj
 0002:00000a00       ??_C@_0BN@LLMKHMNF@JVMTI_ERROR_INVALID_PRIORITY@ 0000000180005a00     libpopframe009.obj
 0002:00000a20       ??_C@_0CB@MBOFKAGB@JVMTI_ERROR_THREAD_NOT_SUSPENDE@ 0000000180005a20     libpopframe009.obj
 0002:00000a48       ??_C@_0BN@FABOLPBI@JVMTI_ERROR_THREAD_SUSPENDED@ 0000000180005a48     libpopframe009.obj
 0002:00000a68       ??_C@_0BN@FDGNOBJM@JVMTI_ERROR_THREAD_NOT_ALIVE@ 0000000180005a68     libpopframe009.obj
 0002:00000a88       ??_C@_0BL@GOBIFKNJ@JVMTI_ERROR_INVALID_OBJECT@ 0000000180005a88     libpopframe009.obj
 0002:00000aa8       ??_C@_0BK@FCMAJPPC@JVMTI_ERROR_INVALID_CLASS@ 0000000180005aa8     libpopframe009.obj
 0002:00000ac8       ??_C@_0BP@IKLLBKEB@JVMTI_ERROR_CLASS_NOT_PREPARED@ 0000000180005ac8     libpopframe009.obj
 0002:00000ae8       ??_C@_0BN@KLPPLKG@JVMTI_ERROR_INVALID_METHODID@ 0000000180005ae8     libpopframe009.obj
 0002:00000b08       ??_C@_0BN@BCEKOKND@JVMTI_ERROR_INVALID_LOCATION@ 0000000180005b08     libpopframe009.obj
 0002:00000b28       ??_C@_0BM@DFDGPME@JVMTI_ERROR_INVALID_FIELDID@ 0000000180005b28     libpopframe009.obj
 0002:00000b48       ??_C@_0BL@NELIEPEC@JVMTI_ERROR_NO_MORE_FRAMES@ 0000000180005b48     libpopframe009.obj
 0002:00000b68       ??_C@_0BJ@BDBECFDM@JVMTI_ERROR_OPAQUE_FRAME@ 0000000180005b68     libpopframe009.obj
 0002:00000b88       ??_C@_0BK@MIIFNLOB@JVMTI_ERROR_TYPE_MISMATCH@ 0000000180005b88     libpopframe009.obj
 0002:00000ba8       ??_C@_0BJ@HPCAOILC@JVMTI_ERROR_INVALID_SLOT@ 0000000180005ba8     libpopframe009.obj
 0002:00000bc8       ??_C@_0BG@CHILOPNI@JVMTI_ERROR_DUPLICATE@ 0000000180005bc8     libpopframe009.obj
 0002:00000be0       ??_C@_0BG@DIEMLHKM@JVMTI_ERROR_NOT_FOUND@ 0000000180005be0     libpopframe009.obj
 0002:00000bf8       ??_C@_0BM@NHMCKHOB@JVMTI_ERROR_INVALID_MONITOR@ 0000000180005bf8     libpopframe009.obj
 0002:00000c18       ??_C@_0BO@PPEDAJGL@JVMTI_ERROR_NOT_MONITOR_OWNER@ 0000000180005c18     libpopframe009.obj
 0002:00000c38       ??_C@_0BG@FCAIPEID@JVMTI_ERROR_INTERRUPT@ 0000000180005c38     libpopframe009.obj
 0002:00000c50       ??_C@_0CB@EGDBNKOI@JVMTI_ERROR_INVALID_CLASS_FORMA@ 0000000180005c50     libpopframe009.obj
 0002:00000c78       ??_C@_0CG@DGKOGIAL@JVMTI_ERROR_CIRCULAR_CLASS_DEFI@ 0000000180005c78     libpopframe009.obj
 0002:00000ca0       ??_C@_0BP@ICEALPKC@JVMTI_ERROR_FAILS_VERIFICATION@ 0000000180005ca0     libpopframe009.obj
 0002:00000cc0       ??_C@_0DC@JDACLMIO@JVMTI_ERROR_UNSUPPORTED_REDEFIN@ 0000000180005cc0     libpopframe009.obj
 0002:00000cf8       ??_C@_0DE@GKDKNOMJ@JVMTI_ERROR_UNSUPPORTED_REDEFIN@ 0000000180005cf8     libpopframe009.obj
 0002:00000d30       ??_C@_0BO@LAFKIOG@JVMTI_ERROR_INVALID_TYPESTATE@ 0000000180005d30     libpopframe009.obj
 0002:00000d50       ??_C@_0DH@INDGCLLB@JVMTI_ERROR_UNSUPPORTED_REDEFIN@ 0000000180005d50     libpopframe009.obj
 0002:00000d88       ??_C@_0DE@NHEOMMGI@JVMTI_ERROR_UNSUPPORTED_REDEFIN@ 0000000180005d88     libpopframe009.obj
 0002:00000dc0       ??_C@_0CA@EKPNJOEP@JVMTI_ERROR_UNSUPPORTED_VERSION@ 0000000180005dc0     libpopframe009.obj
 0002:00000de0       ??_C@_0BN@OFFMAHHL@JVMTI_ERROR_NAMES_DONT_MATCH@ 0000000180005de0     libpopframe009.obj
 0002:00000e00       ??_C@_0DN@HHBBLAKE@JVMTI_ERROR_UNSUPPORTED_REDEFIN@ 0000000180005e00     libpopframe009.obj
 0002:00000e40       ??_C@_0DO@HMBGBGNA@JVMTI_ERROR_UNSUPPORTED_REDEFIN@ 0000000180005e40     libpopframe009.obj
 0002:00000e80       ??_C@_0BP@PBECGKHJ@JVMTI_ERROR_UNMODIFIABLE_CLASS@ 0000000180005e80     libpopframe009.obj
 0002:00000ea0       ??_C@_0BK@CANILEHF@JVMTI_ERROR_NOT_AVAILABLE@ 0000000180005ea0     libpopframe009.obj
 0002:00000ec0       ??_C@_0CE@INJKMEFK@JVMTI_ERROR_MUST_POSSESS_CAPABI@ 0000000180005ec0     libpopframe009.obj
 0002:00000ee8       ??_C@_0BJ@LBFPFPDM@JVMTI_ERROR_NULL_POINTER@ 0000000180005ee8     libpopframe009.obj
 0002:00000f08       ??_C@_0BP@CHJPNNEM@JVMTI_ERROR_ABSENT_INFORMATION@ 0000000180005f08     libpopframe009.obj
 0002:00000f28       ??_C@_0BP@OMFMNLC@JVMTI_ERROR_INVALID_EVENT_TYPE@ 0000000180005f28     libpopframe009.obj
 0002:00000f48       ??_C@_0BN@BIBNPHHO@JVMTI_ERROR_ILLEGAL_ARGUMENT@ 0000000180005f48     libpopframe009.obj
 0002:00000f68       ??_C@_0BK@KKNDHDCE@JVMTI_ERROR_NATIVE_METHOD@ 0000000180005f68     libpopframe009.obj
 0002:00000f88       ??_C@_0BK@PMKCFHAE@JVMTI_ERROR_OUT_OF_MEMORY@ 0000000180005f88     libpopframe009.obj
 0002:00000fa8       ??_C@_0BK@NNJBDMNB@JVMTI_ERROR_ACCESS_DENIED@ 0000000180005fa8     libpopframe009.obj
 0002:00000fc8       ??_C@_0BI@GHECLMNC@JVMTI_ERROR_WRONG_PHASE@ 0000000180005fc8     libpopframe009.obj
 0002:00000fe0       ??_C@_0BF@OLIHJOII@JVMTI_ERROR_INTERNAL@ 0000000180005fe0     libpopframe009.obj
 0002:00000ff8       ??_C@_0BO@EOHGKJHI@JVMTI_ERROR_UNATTACHED_THREAD@ 0000000180005ff8     libpopframe009.obj
 0002:00001018       ??_C@_0CA@LKHFDACL@JVMTI_ERROR_INVALID_ENVIRONMENT@ 0000000180006018     libpopframe009.obj
 0002:00001038       ??_C@_0BA@MMFHLOKK@?$DMunknown?5error?$DO@ 0000000180006038     libpopframe009.obj
 0002:00001048       ??_C@_0CF@CBHOKDB@throwable?5?$DN?5jni?9?$DOExceptionOccur@ 0000000180006048     libpopframe009.obj
 0002:00001070       ??_C@_03OFAPEBGM@?$CFs?6@  0000000180006070     libpopframe009.obj
 0002:00001078       ??_C@_0DM@LPIGEGNJ@s?2test?2hotspot?2jtreg?2vmTestbase@ 0000000180006078     libpopframe009.obj
 0002:000010b8       ??_C@_0CC@NFCNPEPK@Exception?5in?5JNI?5call?5?$CIcleared?$CJ@ 00000001800060b8     libpopframe009.obj
 0002:000010e0       ??_C@_0BJ@IBAKFIKF@jni?9?$DOExceptionDescribe?$CI?$CJ@ 00000001800060e0     libpopframe009.obj
 0002:00001100       ??_C@_0BG@GGKALKMH@jni?9?$DOExceptionClear?$CI?$CJ@ 0000000180006100     libpopframe009.obj
 0002:00001118       ??_C@_0CF@JMGFGJLJ@?$CD?5?5?5verified?5JNI?5assertion?5is?5F@ 0000000180006118     libpopframe009.obj
 0002:00001140       ??_C@_0CB@MLNJNCLJ@?5?5jvmti?5error?3?5code?$DN?$CFd?0?5name?$DN?$CFs@ 0000000180006140     libpopframe009.obj
 0002:00001168       ??_C@_0CD@OHBGDKMK@?$CD?5?5?5jvmti?5error?3?5code?$DN?$CFd?0?5name?$DN@ 0000000180006168     libpopframe009.obj
 0002:00001190       ??_C@_0CG@JNNCGPHB@?$CD?5?5?5error?5expected?3?5code?$DN?$CFd?0?5na@ 0000000180006190     libpopframe009.obj
 0002:000011c0       ??_C@_0EB@IMGKPCGE@?$CIstr_obj?5?$DN?5jni?9?$DONewStringUTF?$CIco@ 00000001800061c0     libpopframe009.obj
 0002:00001210       ??_C@_0EA@HFOGGBCC@s?2test?2hotspot?2jtreg?2vmTestbase@ 0000000180006210     libpopframe009.obj
 0002:00001250       ??_C@_0CO@HJKAMPK@?$CIGetFrameLocation?$CJ?5unexpected?5e@ 0000000180006250     libpopframe009.obj
 0002:00001280       ??_C@_0CK@GNODJBHO@?$CIResumeThread?$CJ?5unexpected?5error@ 0000000180006280     libpopframe009.obj
 0002:000012b0       ??_C@_0CL@KLNIBDFF@?$CISuspendThread?$CJ?5unexpected?5erro@ 00000001800062b0     libpopframe009.obj
 0002:000012dc       ??_C@_05KKCIMGE@error@     00000001800062dc     libpopframe009.obj
 0002:000012e8       ??_C@_0CJ@JACLEAA@Test?5failed?5by?5setFailStatus?$CI?$CJ?4@ 00000001800062e8     libpopframe009.obj
 0002:00001320       ??_C@_0EA@PNBCDMOA@s?2test?2hotspot?2jtreg?2vmTestbase@ 0000000180006320     libpopframe009.obj
 0002:00001360       ??_C@_0DI@ILAHDLMP@?$CI?$CKagentThreadProc?$CJ?$CIjvmti_env?0?5a@ 0000000180006360     libpopframe009.obj
 0002:00001398       ??_C@_0BD@KDBALNLB@JVMTI?5agent?5thread@ 0000000180006398     libpopframe009.obj
 0002:000013b0       ??_C@_0BB@NOKBFPFO@java?1lang?1Thread@ 00000001800063b0     libpopframe009.obj
 0002:000013c4       ??_C@_06FALKBLGB@?$DMinit?$DO@ 00000001800063c4     libpopframe009.obj
 0002:000013d0       ??_C@_0BG@IKDDPPGD@?$CILjava?1lang?1String?$DL?$CJV@ 00000001800063d0     libpopframe009.obj
 0002:000013f0       ??_C@_0EB@IFJBFEKC@?$CIthreadClass?5?$DN?5jni_env?9?$DOFindCla@ 00000001800063f0     libpopframe009.obj
 0002:00001440       ??_C@_0GF@FGFIBKKL@?$CIthreadCtor?5?$DN?5jni_env?9?$DOGetMetho@ 0000000180006440     libpopframe009.obj
 0002:000014a8       ??_C@_0DN@NCPDJLOG@?$CIthreadName?5?$DN?5jni_env?9?$DONewStrin@ 00000001800064a8     libpopframe009.obj
 0002:000014f0       ??_C@_0FE@PFKODBGC@?$CIthreadObject?5?$DN?5jni_env?9?$DONewObj@ 00000001800064f0     libpopframe009.obj
 0002:00001550       ??_C@_0ED@HOBAHHJI@?$CIthreadGlobalRef?5?$DN?5jni_env?9?$DONew@ 0000000180006550     libpopframe009.obj
 0002:000015a0       ??_C@_0FN@HNJJAHFC@jvmti_env?9?$DORunAgentThread?$CIagent@ 00000001800065a0     libpopframe009.obj
 0002:00001600       ??_C@_0EA@MOJDNKDF@Debuggee?5status?5sync?5aborted?5be@ 0000000180006600     libpopframe009.obj
 0002:00001640       ??_C@_0EA@EEOEJAEN@status?5?$DN?5syncDebuggeeStatus?$CIjni@ 0000000180006640     libpopframe009.obj
 0002:00001680       ??_C@_0BL@JBCFNBMB@nsk_jvmti_resetAgentData?$CI?$CJ@ 0000000180006680     libpopframe009.obj
 0002:0000169c       ??_C@_04DIFHPCLD@?$CII?$CJI@ 000000018000669c     libpopframe009.obj
 0002:000016b0       ??_C@_0EL@LPBEELIP@s?2test?2hotspot?2jtreg?2vmTestbase@ 00000001800066b0     libpopframe009.obj
 0002:00001700       ??_C@_0CK@JDAMFDMJ@jvmti?9?$DOSetTag?$CIo?0?5tag?$CJ?5?$DN?$DN?5JVMTI_@ 0000000180006700     libpopframe009.obj
 0002:00001730       ??_C@_0CC@DAMNHKNI@Can?8t?5set?5tag?5?$CFli?5for?5object?5?$CFl@ 0000000180006730     libpopframe009.obj
 0002:00001758       ??_C@_0DL@HAJPNKEF@jvmti?9?$DOGetObjectHashCode?$CIo?0?5?$CGha@ 0000000180006758     libpopframe009.obj
 0002:00001798       ??_C@_0BL@JFPIEOBF@Can?8t?5get?5hash?5object?5?$CFlx?6@ 0000000180006798     libpopframe009.obj
 0002:000017b8       ??_C@_0BG@DICPHBKN@setTag?3?5?$CF08x?5?$DM?9?5?$CF?53li@ 00000001800067b8     libpopframe009.obj
 0002:000017d0       ??_C@_0DH@FCEEBDMJ@?$CIs?5?$DN?5jni?9?$DOGetStringUTFChars?$CIsIn@ 00000001800067d0     libpopframe009.obj
 0002:00001808       ??_C@_0BJ@OKKGHDCN@Can?8t?5get?5string?5at?5?$CF?$CDp?6@ 0000000180006808     libpopframe009.obj
 0002:00001828       ??_C@_0BP@EKFLGGFJ@Can?8t?5get?5string?5at?5?$CF?$CDp?3?5null?6@ 0000000180006828     libpopframe009.obj
 0002:00001848       ??_C@_06ICODBHCL@?5?1?1?5?$CFs@ 0000000180006848     libpopframe009.obj
 0002:00001850       ??_C@_0DB@KGFPLEGO@?$CIr?5?$DN?5jvmti?9?$DOGetTag?$CIo?0?5?$CGtag?$CJ?$CJ?5?$DN?$DN@ 0000000180006850     libpopframe009.obj
 0002:00001888       ??_C@_0CO@PDAGBCGJ@Can?8t?5GetTag?5for?5object?5?$CFlx?4?5Re@ 0000000180006888     libpopframe009.obj
 0002:000018b8       ??_C@_0CH@HPEODOHC@TEST_BUG?3?5Max?4?5number?5of?5refs?5r@ 00000001800068b8     libpopframe009.obj
 0002:000018e0       ??_C@_0DI@PHFCABIM@?$CIr?5?$DN?5jvmti?9?$DOGetTag?$CIfrom?0?5?$CGtagFr@ 00000001800068e0     libpopframe009.obj
 0002:00001918       ??_C@_0DI@MDEGFNKD@TEST_BUG?3?5Can?8t?5GetTag?5for?5obje@ 0000000180006918     libpopframe009.obj
 0002:00001950       ??_C@_0DE@MLELJAHM@?$CIr?5?$DN?5jvmti?9?$DOGetTag?$CIto?0?5?$CGtagTo?$CJ?$CJ@ 0000000180006950     libpopframe009.obj
 0002:00001984       ??_C@_03GAEACAIP@?$CI?$CJV@ 0000000180006984     libpopframe009.obj
 0002:00001988       ??_C@_0CI@ODAHCOFC@bp?3?5don?8t?5know?5where?5we?5get?5cal@ 0000000180006988     libpopframe009.obj
 0002:000019b0       ??_C@_0CM@ELOAFJPP@step?3?5Cannot?5enter?5breakpointLo@ 00000001800069b0     libpopframe009.obj
 0002:000019e0       ??_C@_0BD@KBBLJLHF@?$DO?$DO?$DO?5breakpoint?5?$CFd?6@ 00000001800069e0     libpopframe009.obj
 0002:000019f8       ??_C@_0CL@JHEKLOBF@step?3?5Cannot?5wait?5breakpointLoc@ 00000001800069f8     libpopframe009.obj
 0002:00001a28       ??_C@_0CN@MNGFMGHL@?$CIClearBreakpoint?$CJ?5unexpected?5er@ 0000000180006a28     libpopframe009.obj
 0002:00001a58       ??_C@_0CL@NEHENFIE@step?3?5Cannot?5exit?5breakpointLoc@ 0000000180006a58     libpopframe009.obj
 0002:00001a88       ??_C@_0CC@NJGDDDCL@?$DO?$DO?$DO?5poped?5?$CFd?5frames?5till?5?$CCrun?$CI?$CJ@ 0000000180006a88     libpopframe009.obj
 0002:00001ab0       ??_C@_0CJ@FPJJBCFO@step?3?5Cannot?5enter?5suspendLock?3@ 0000000180006ab0     libpopframe009.obj
 0002:00001ae0       ??_C@_0CK@LIACFPNH@step?3?5Cannot?5enter?5popFrameLock@ 0000000180006ae0     libpopframe009.obj
 0002:00001b10       ??_C@_0CL@HGMOBJIL@step?3?5Cannot?5notify?5popFrameLoc@ 0000000180006b10     libpopframe009.obj
 0002:00001b40       ??_C@_0CJ@GEIGILGN@step?3?5Cannot?5exit?5popFrameLock?3@ 0000000180006b40     libpopframe009.obj
 0002:00001b70       ??_C@_0CI@JGEKCKPE@step?3?5Cannot?5wait?5suspendLock?3?5@ 0000000180006b70     libpopframe009.obj
 0002:00001b98       ??_C@_0CI@NEAGHHA@step?3?5Cannot?5exit?5suspendLock?3?5@ 0000000180006b98     libpopframe009.obj
 0002:00001bc0       ??_C@_09OPJEJKBL@printdump@ 0000000180006bc0     libpopframe009.obj
 0002:00001bd0       ??_C@_0CJ@KCDEKOCJ@Wrong?5result?5of?5a?5valid?5call?5to@ 0000000180006bd0     libpopframe009.obj
 0002:00001c00       ??_C@_0DG@LAJPGIIE@?$CIGetPotentialCapabilities?$CJ?5unex@ 0000000180006c00     libpopframe009.obj
 0002:00001c38       ??_C@_0CN@LKPEOJPO@?$CIAddCapabilities?$CJ?5unexpected?5er@ 0000000180006c38     libpopframe009.obj
 0002:00001c68       ??_C@_0CN@BCCBOHCH@?$CIGetCapabilities?$CJ?5unexpected?5er@ 0000000180006c68     libpopframe009.obj
 0002:00001c98       ??_C@_0CG@MCCDAOGE@Warning?3?5PopFrame?5is?5not?5implem@ 0000000180006c98     libpopframe009.obj
 0002:00001cc0       ??_C@_0CM@FEKJDMLD@Warning?3?5suspend?1resume?5is?5not?5@ 0000000180006cc0     libpopframe009.obj
 0002:00001cf0       ??_C@_0CP@IMINGNLL@?$CISetEventCallbacks?$CJ?5unexpected?5@ 0000000180006cf0     libpopframe009.obj
 0002:00001d20       ??_C@_0DN@NCDMFLGJ@Warning?3?5Breakpoint?5or?5SingleSt@ 0000000180006d20     libpopframe009.obj
 0002:00001d60       ??_C@_0CH@CDOJMNAO@JVMTI?5client?5was?5not?5properly?5l@ 0000000180006d60     libpopframe009.obj
 0002:00001d88       ??_C@_0L@GIHILDI@checkPoint@ 0000000180006d88     libpopframe009.obj
 0002:00001d98       ??_C@_0CN@GIADEMBI@Cannot?5find?5Method?5ID?5for?5metho@ 0000000180006d98     libpopframe009.obj
 0002:00001dc8       ??_C@_0BA@FAKBMKOJ@Breakpoint?5Lock@ 0000000180006dc8     libpopframe009.obj
 0002:00001dd8       ??_C@_0CH@DOPAACCG@Cannot?5create?5breakpointLock?3?5?$CF@ 0000000180006dd8     libpopframe009.obj
 0002:00001e00       ??_C@_0CL@GMOLCHIJ@?$CISetBreakpoint?$CJ?5unexpected?5erro@ 0000000180006e00     libpopframe009.obj
 0002:00001e30       ??_C@_0CM@NEGFNKGE@Failed?5to?5enable?5BREAKPOINT?5eve@ 0000000180006e30     libpopframe009.obj
 0002:00001e60       ??_C@_0CG@LNOCPLAB@?$CIPopFrame?$CJ?5unexpected?5error?3?5?$CFs@ 0000000180006e60     libpopframe009.obj
 0002:00001e88       ??_C@_0CD@CHOAPNEP@Cannot?5wait?5popFrameLock?3?5?$CFs?5?$CI?$CF@ 0000000180006e88     libpopframe009.obj
 0002:00001eb0       ??_C@_0CD@PGLBCJAI@Cannot?5enter?5suspendLock?3?5?$CFs?5?$CI?$CF@ 0000000180006eb0     libpopframe009.obj
 0002:00001ed8       ??_C@_0CE@HAJKANND@Cannot?5notify?5suspendLock?3?5?$CFs?5?$CI@ 0000000180006ed8     libpopframe009.obj
 0002:00001f00       ??_C@_0CC@JJNFGCJM@Cannot?5exit?5suspendLock?3?5?$CFs?5?$CI?$CFd@ 0000000180006f00     libpopframe009.obj
 0002:00001f28       ??_C@_0P@POHCNBHB@Pop?5Frame?5Lock@ 0000000180006f28     libpopframe009.obj
 0002:00001f38       ??_C@_0CF@CKBNDFFM@Cannot?5create?5popFrameLock?3?5?$CFs?5@ 0000000180006f38     libpopframe009.obj
 0002:00001f60       ??_C@_0BK@BNKNDDLD@?$DO?$DO?$DO?5waiting?5breakpoint?51?6@ 0000000180006f60     libpopframe009.obj
 0002:00001f80       ??_C@_0CE@DKKDIDCN@Cannot?5enter?5popFrameLock?3?5?$CFs?5?$CI@ 0000000180006f80     libpopframe009.obj
 0002:00001fa8       ??_C@_0CD@MNKOLADL@Cannot?5exit?5popFrameLock?3?5?$CFs?5?$CI?$CF@ 0000000180006fa8     libpopframe009.obj
 0002:00001fd0       ??_C@_0CG@CKNGEMJG@Cannot?5enter?5breakpointLock?3?5?$CFs@ 0000000180006fd0     libpopframe009.obj
 0002:00001ff8       ??_C@_0CH@PGFOIOCH@Cannot?5notify?5breakpointLock?3?5?$CF@ 0000000180006ff8     libpopframe009.obj
 0002:00002020       ??_C@_0CF@IJJOGPFK@Cannot?5exit?5breakpointLock?3?5?$CFs?5@ 0000000180007020     libpopframe009.obj
 0002:00002048       ??_C@_09JOONICCG@fibonacci@ 0000000180007048     libpopframe009.obj
 0002:00002058       ??_C@_0CN@MNOAKOOJ@Cannot?5get?5method?5ID?5for?5method@ 0000000180007058     libpopframe009.obj
 0002:00002088       ??_C@_0CD@MAPGAMMD@Cannot?5get?5class?5of?5thread?5obje@ 0000000180007088     libpopframe009.obj
 0002:000020ac       ??_C@_03LGMJKEGG@run@      00000001800070ac     libpopframe009.obj
 0002:000020b0       ??_C@_0CA@HCOMBIJN@Cannot?5get?5method?5ID?5for?5?$CCrun?$CC?6@ 00000001800070b0     libpopframe009.obj
 0002:000020d0       ??_C@_0CB@HEIAOBNL@?$DO?$DO?$DO?5catching?5method?5?$CCfibonacci?$CC@ 00000001800070d0     libpopframe009.obj
 0002:000020f8       ??_C@_0BA@LHGLOEPK@?$DO?$DO?$DO?5?$CFd?3?5?$CC?$CFs?$CFs?$CC?6@ 00000001800070f8     libpopframe009.obj
 0002:00002108       ??_C@_0CE@FMDJGKKD@Cannot?5enable?5single?5step?3?5?$CFs?5?$CI@ 0000000180007108     libpopframe009.obj
 0002:00002130       ??_C@_0N@PALFCLOG@Suspend?5Lock@ 0000000180007130     libpopframe009.obj
 0002:00002140       ??_C@_0CE@JCHNACJC@Cannot?5create?5suspendLock?3?5?$CFs?5?$CI@ 0000000180007140     libpopframe009.obj
 0002:00002168       ??_C@_0BE@GDJPJMM@?$DO?$DO?$DO?5popping?5frames?6@ 0000000180007168     libpopframe009.obj
 0002:00002180       ??_C@_0CF@OAOLHEMH@Cannot?5disable?5single?5step?3?5?$CFs?5@ 0000000180007180     libpopframe009.obj
 0002:000021a8       ??_C@_0CI@JPKFBKLB@Warning?3?5method?5?$CCfibonacci?$CC?5was@ 00000001800071a8     libpopframe009.obj
 0002:000021d0       ??_C@_0BK@BPOLINOK@?$DO?$DO?$DO?5waiting?5breakpoint?52?6@ 00000001800071d0     libpopframe009.obj
 0002:00002200       ??_C@_1EC@JIJBPKFM@?$AAa?$AAp?$AAi?$AA?9?$AAm?$AAs?$AA?9?$AAw?$AAi?$AAn?$AA?9?$AAc?$AAo?$AAr?$AAe@ 0000000180007200     MSVCRT:thread_safe_statics.obj
 0002:00002248       ??_C@_1BK@MGMFAEKH@?$AAk?$AAe?$AAr?$AAn?$AAe?$AAl?$AA3?$AA2?$AA?4?$AAd?$AAl?$AAl@ 0000000180007248     MSVCRT:thread_safe_statics.obj
 0002:00002268       ??_C@_0BJ@JEBJOJFJ@SleepConditionVariableCS@ 0000000180007268     MSVCRT:thread_safe_statics.obj
 0002:00002288       ??_C@_0BJ@PGPPEPCC@WakeAllConditionVariable@ 0000000180007288     MSVCRT:thread_safe_statics.obj
 0002:000022a8       _pDefaultRawDllMain        00000001800072a8     MSVCRT:dll_dllmain.obj
 0002:000022a8       _pRawDllMain               00000001800072a8     MSVCRT:dll_dllmain.obj
 0002:000022b0       __xmm@ffffffffffffffffffffffffffffffff 00000001800072b0     MSVCRT:utility.obj
 0002:000022c0       _load_config_used          00000001800072c0     MSVCRT:loadcfg.obj
 0002:00002480       _tls_used                  0000000180007480     MSVCRT:tlssup.obj
 0002:000024a8       __volatile_metadata        00000001800074a8     <linker-defined>
 0002:00002868       __rtc_iaa                  0000000180007868     MSVCRT:initsect.obj
 0002:00002870       __rtc_izz                  0000000180007870     MSVCRT:initsect.obj
 0002:00002878       __rtc_taa                  0000000180007878     MSVCRT:initsect.obj
 0002:00002880       __rtc_tzz                  0000000180007880     MSVCRT:initsect.obj
 0002:00002888       _tls_start                 0000000180007888     MSVCRT:tlssup.obj
 0002:0000288c       _Init_thread_epoch         000000018000788c     MSVCRT:thread_safe_statics.obj
 0002:00002890       _tls_end                   0000000180007890     MSVCRT:tlssup.obj
 0002:00002f70       __IMPORT_DESCRIPTOR_KERNEL32 0000000180007f70     kernel32:KERNEL32.dll
 0002:00002f84       __IMPORT_DESCRIPTOR_VCRUNTIME140 0000000180007f84     vcruntime:VCRUNTIME140.dll
 0002:00002f98       __IMPORT_DESCRIPTOR_api-ms-win-crt-runtime-l1-1-0 0000000180007f98     ucrt:api-ms-win-crt-runtime-l1-1-0.dll
 0002:00002fac       __IMPORT_DESCRIPTOR_api-ms-win-crt-stdio-l1-1-0 0000000180007fac     ucrt:api-ms-win-crt-stdio-l1-1-0.dll
 0002:00002fc0       __IMPORT_DESCRIPTOR_api-ms-win-crt-string-l1-1-0 0000000180007fc0     ucrt:api-ms-win-crt-string-l1-1-0.dll
 0002:00002fd4       __NULL_IMPORT_DESCRIPTOR   0000000180007fd4     kernel32:KERNEL32.dll
 0003:00000030       _Init_global_epoch         0000000180009030     MSVCRT:thread_safe_statics.obj
 0003:00000040       __security_cookie          0000000180009040     MSVCRT:gs_cookie.obj
 0003:00000048       __security_cookie_complement 0000000180009048     MSVCRT:gs_cookie.obj
 0003:00000050       __scrt_native_dllmain_reason 0000000180009050     MSVCRT:utility.obj
 0003:00000058       __isa_available            0000000180009058     MSVCRT:cpu_disp.obj
 0003:0000005c       __isa_enabled              000000018000905c     MSVCRT:cpu_disp.obj
 0003:00000060       __memset_fast_string_threshold 0000000180009060     MSVCRT:cpu_disp.obj
 0003:00000068       __memset_nt_threshold      0000000180009068     MSVCRT:cpu_disp.obj
 0003:00000070       __scrt_ucrt_dll_is_in_use  0000000180009070     MSVCRT:ucrt_stubs.obj
 0003:00000080       g_wrongHeapCallbacks       0000000180009080     libpopframe009.obj
 0003:00000100       g_szTagInfo                0000000180009100     libpopframe009.obj
 0003:00002040       g_tagFlags                 000000018000b040     libpopframe009.obj
 0003:00002428       g_refsToVerifyCnt          000000018000b428     libpopframe009.obj
 0003:0000242c       g_fakeUserData             000000018000b42c     libpopframe009.obj
 0003:00002430       g_tagVisitCount            000000018000b430     libpopframe009.obj
 0003:000033d0       g_refsToVerify             000000018000c3d0     libpopframe009.obj
 0003:0001aad0       g_userDataError            0000000180023ad0     libpopframe009.obj
 0003:0001ade8       ?_OptionsStorage@?1??__local_stdio_printf_options@@9@4_KA 0000000180023de8     libpopframe009.obj
 0003:0001b3a8       _tls_index                 00000001800243a8     MSVCRT:tlssup.obj
 0003:0001b3b0       __scrt_current_native_startup_state 00000001800243b0     MSVCRT:utility.obj
 0003:0001b3b8       __scrt_native_startup_lock 00000001800243b8     MSVCRT:utility.obj
 0003:0001b3f8       __scrt_debugger_hook_flag  00000001800243f8     MSVCRT:utility_desktop.obj
 0003:0001b400       ?__type_info_root_node@@3U__type_info_node@@A 0000000180024400     MSVCRT:tncleanup.obj
 0003:0001b410       ?_OptionsStorage@?1??__local_stdio_scanf_options@@9@4_KA 0000000180024410     MSVCRT:default_local_stdio_options.obj
 0003:0001b418       __favor                    0000000180024418     MSVCRT:cpu_disp.obj
 0003:0001b420       __dyn_tls_init_callback    0000000180024420     <common>

 entry point at        0001:00003150

 Static symbols

 0000:fffd9000       .debug$S                   0000000180000000     popframe009.exp
 0000:fffd9000       .debug$S                   0000000180000000     vcruntime:VCRUNTIME140.dll
 0000:fffd9000       .debug$S                   0000000180000000     vcruntime:VCRUNTIME140.dll
 0000:fffd9000       .debug$S                   0000000180000000     vcruntime:VCRUNTIME140.dll
 0000:fffd9000       .debug$S                   0000000180000000     vcruntime:VCRUNTIME140.dll
 0000:fffd9000       .debug$S                   0000000180000000     vcruntime:VCRUNTIME140.dll
 0000:fffd9000       .debug$S                   0000000180000000     vcruntime:VCRUNTIME140.dll
 0000:fffd9000       .debug$S                   0000000180000000     vcruntime:VCRUNTIME140.dll
 0000:fffd9000       .debug$S                   0000000180000000     ucrt:api-ms-win-crt-convert-l1-1-0.dll
 0002:ffffb000       .idata$6                   0000000180000000     ucrt:api-ms-win-crt-convert-l1-1-0.dll
 0000:fffd9000       .debug$S                   0000000180000000     ucrt:api-ms-win-crt-heap-l1-1-0.dll
 0000:fffd9000       .debug$S                   0000000180000000     ucrt:api-ms-win-crt-heap-l1-1-0.dll
 0000:fffd9000       .debug$S                   0000000180000000     ucrt:api-ms-win-crt-heap-l1-1-0.dll
 0000:fffd9000       .debug$S                   0000000180000000     ucrt:api-ms-win-crt-heap-l1-1-0.dll
 0002:ffffb000       .idata$6                   0000000180000000     ucrt:api-ms-win-crt-heap-l1-1-0.dll
 0000:fffd9000       .debug$S                   0000000180000000     ucrt:api-ms-win-crt-runtime-l1-1-0.dll
 0000:fffd9000       .debug$S                   0000000180000000     ucrt:api-ms-win-crt-runtime-l1-1-0.dll
 0000:fffd9000       .debug$S                   0000000180000000     ucrt:api-ms-win-crt-runtime-l1-1-0.dll
 0000:fffd9000       .debug$S                   0000000180000000     ucrt:api-ms-win-crt-runtime-l1-1-0.dll
 0000:fffd9000       .debug$S                   0000000180000000     ucrt:api-ms-win-crt-runtime-l1-1-0.dll
 0000:fffd9000       .debug$S                   0000000180000000     ucrt:api-ms-win-crt-runtime-l1-1-0.dll
 0000:fffd9000       .debug$S                   0000000180000000     ucrt:api-ms-win-crt-runtime-l1-1-0.dll
 0000:fffd9000       .debug$S                   0000000180000000     ucrt:api-ms-win-crt-runtime-l1-1-0.dll
 0000:fffd9000       .debug$S                   0000000180000000     ucrt:api-ms-win-crt-runtime-l1-1-0.dll
 0000:fffd9000       .debug$S                   0000000180000000     ucrt:api-ms-win-crt-runtime-l1-1-0.dll
 0000:fffd9000       .debug$S                   0000000180000000     ucrt:api-ms-win-crt-runtime-l1-1-0.dll
 0000:fffd9000       .debug$S                   0000000180000000     ucrt:api-ms-win-crt-runtime-l1-1-0.dll
 0000:fffd9000       .debug$S                   0000000180000000     ucrt:api-ms-win-crt-runtime-l1-1-0.dll
 0000:fffd9000       .debug$S                   0000000180000000     ucrt:api-ms-win-crt-runtime-l1-1-0.dll
 0000:fffd9000       .debug$S                   0000000180000000     ucrt:api-ms-win-crt-runtime-l1-1-0.dll
 0000:fffd9000       .debug$S                   0000000180000000     ucrt:api-ms-win-crt-runtime-l1-1-0.dll
 0000:fffd9000       .debug$S                   0000000180000000     ucrt:api-ms-win-crt-stdio-l1-1-0.dll
 0000:fffd9000       .debug$S                   0000000180000000     ucrt:api-ms-win-crt-stdio-l1-1-0.dll
 0000:fffd9000       .debug$S                   0000000180000000     ucrt:api-ms-win-crt-stdio-l1-1-0.dll
 0000:fffd9000       .debug$S                   0000000180000000     ucrt:api-ms-win-crt-stdio-l1-1-0.dll
 0000:fffd9000       .debug$S                   0000000180000000     ucrt:api-ms-win-crt-stdio-l1-1-0.dll
 0000:fffd9000       .debug$S                   0000000180000000     ucrt:api-ms-win-crt-stdio-l1-1-0.dll
 0000:fffd9000       .debug$S                   0000000180000000     ucrt:api-ms-win-crt-stdio-l1-1-0.dll
 0000:fffd9000       .debug$S                   0000000180000000     ucrt:api-ms-win-crt-stdio-l1-1-0.dll
 0000:fffd9000       .debug$S                   0000000180000000     ucrt:api-ms-win-crt-stdio-l1-1-0.dll
 0000:fffd9000       .debug$S                   0000000180000000     ucrt:api-ms-win-crt-stdio-l1-1-0.dll
 0000:fffd9000       .debug$S                   0000000180000000     ucrt:api-ms-win-crt-string-l1-1-0.dll
 0000:fffd9000       .debug$S                   0000000180000000     ucrt:api-ms-win-crt-string-l1-1-0.dll
 0000:fffd9000       .debug$S                   0000000180000000     ucrt:api-ms-win-crt-string-l1-1-0.dll
 0000:fffd9000       .debug$S                   0000000180000000     ucrt:api-ms-win-crt-string-l1-1-0.dll
 0000:fffd9000       .debug$S                   0000000180000000     ucrt:api-ms-win-crt-string-l1-1-0.dll
 0000:fffd9000       .debug$S                   0000000180000000     ucrt:api-ms-win-crt-string-l1-1-0.dll
 0000:fffd9000       .debug$S                   0000000180000000     ucrt:api-ms-win-crt-string-l1-1-0.dll
 0000:fffd9000       .debug$S                   0000000180000000     ucrt:api-ms-win-crt-string-l1-1-0.dll
 0000:fffd9000       .debug$S                   0000000180000000     kernel32:KERNEL32.dll
 0000:fffd9000       .debug$S                   0000000180000000     kernel32:KERNEL32.dll
 0000:fffd9000       .debug$S                   0000000180000000     kernel32:KERNEL32.dll
 0000:fffd9000       .debug$S                   0000000180000000     kernel32:KERNEL32.dll
 0000:fffd9000       .debug$S                   0000000180000000     kernel32:KERNEL32.dll
 0000:fffd9000       .debug$S                   0000000180000000     kernel32:KERNEL32.dll
 0000:fffd9000       .debug$S                   0000000180000000     kernel32:KERNEL32.dll
 0000:fffd9000       .debug$S                   0000000180000000     kernel32:KERNEL32.dll
 0000:fffd9000       .debug$S                   0000000180000000     kernel32:KERNEL32.dll
 0000:fffd9000       .debug$S                   0000000180000000     kernel32:KERNEL32.dll
 0000:fffd9000       .debug$S                   0000000180000000     kernel32:KERNEL32.dll
 0000:fffd9000       .debug$S                   0000000180000000     kernel32:KERNEL32.dll
 0000:fffd9000       .debug$S                   0000000180000000     kernel32:KERNEL32.dll
 0000:fffd9000       .debug$S                   0000000180000000     kernel32:KERNEL32.dll
 0000:fffd9000       .debug$S                   0000000180000000     kernel32:KERNEL32.dll
 0000:fffd9000       .debug$S                   0000000180000000     kernel32:KERNEL32.dll
 0000:fffd9000       .debug$S                   0000000180000000     kernel32:KERNEL32.dll
 0000:fffd9000       .debug$S                   0000000180000000     kernel32:KERNEL32.dll
 0000:fffd9000       .debug$S                   0000000180000000     kernel32:KERNEL32.dll
 0000:fffd9000       .debug$S                   0000000180000000     kernel32:KERNEL32.dll
 0000:fffd9000       .debug$S                   0000000180000000     kernel32:KERNEL32.dll
 0000:fffd9000       .debug$S                   0000000180000000     kernel32:KERNEL32.dll
 0000:fffd9000       .debug$S                   0000000180000000     kernel32:KERNEL32.dll
 0000:fffd9000       .debug$S                   0000000180000000     kernel32:KERNEL32.dll
 0000:fffd9000       .debug$S                   0000000180000000     kernel32:KERNEL32.dll
 0000:fffd9000       .debug$S                   0000000180000000     kernel32:KERNEL32.dll
 0000:fffd9000       .debug$S                   0000000180000000     kernel32:KERNEL32.dll
 0000:fffd9000       .debug$S                   0000000180000000     kernel32:KERNEL32.dll
 0001:00001b6c       addRefToVerify             0000000180002b6c f   libpopframe009.obj
 0001:00001bd8       agentThreadWrapper         0000000180002bd8 f   libpopframe009.obj
 0001:00001dc8       file_basename              0000000180002dc8 f   libpopframe009.obj
 0001:00002630       startAgentThreadWrapper    0000000180003630 f   libpopframe009.obj
 0001:00002970       syncDebuggeeStatus         0000000180003970 f   libpopframe009.obj
 0001:00002c10       capture_previous_context   0000000180003c10 f   MSVCRT:gs_report.obj
 0001:00002c84       ?__scrt_initialize_thread_safe_statics@@YAHXZ 0000000180003c84 f   MSVCRT:thread_safe_statics.obj
 0001:00002d54       ?__scrt_uninitialize_thread_safe_statics@@YAXXZ 0000000180003d54 f   MSVCRT:thread_safe_statics.obj
 0001:00002e00       $$000000                   0000000180003e00     MSVCRT:amdsecgs.obj
 0001:00002e30       ?dllmain_crt_dispatch@@YAHQEAUHINSTANCE__@@KQEAX@Z 0000000180003e30 f   MSVCRT:dll_dllmain.obj
 0001:00002e80       ?dllmain_crt_process_attach@@YAHQEAUHINSTANCE__@@QEAX@Z 0000000180003e80 f   MSVCRT:dll_dllmain.obj
 0001:00002f98       ?dllmain_crt_process_detach@@YAH_N@Z 0000000180003f98 f   MSVCRT:dll_dllmain.obj
 0001:0000301c       ?dllmain_dispatch@@YAHQEAUHINSTANCE__@@KQEAX@Z 000000018000401c f   MSVCRT:dll_dllmain.obj
 0001:00003a30       $$000000                   0000000180004a30     MSVCRT:guard_dispatch.obj
 0001:00003a50       $$000000                   0000000180004a50     MSVCRT:guard_xfg_dispatch.obj
 0001:00003a66       ?fin$0@?0??dllmain_crt_process_attach@@YAHQEAUHINSTANCE__@@QEAX@Z@4HA 0000000180004a66 f   MSVCRT:dll_dllmain.obj
 0001:00003a7d       ?fin$0@?0??dllmain_crt_process_detach@@YAH_N@Z@4HA 0000000180004a7d f   MSVCRT:dll_dllmain.obj
 0001:00003a96       ?fin$1@?0??dllmain_crt_process_detach@@YAH_N@Z@4HA 0000000180004a96 f   MSVCRT:dll_dllmain.obj
 0001:00003aaa       ?filt$0@?0??dllmain_dispatch@@YAHQEAUHINSTANCE__@@KQEAX@Z@4HA 0000000180004aaa f   MSVCRT:dll_dllmain.obj
 0001:00003ae0       __scrt_is_nonwritable_in_current_image$filt$0 0000000180004ae0 f   MSVCRT:utility.obj
 0002:000001e8       ?__scrt_initialize_tss_var@@3P6AHXZEA 00000001800051e8     MSVCRT:thread_safe_statics.obj
 0002:00000310       ?opcLengths@@3QBEB         0000000180005310     libpopframe009.obj
 0002:000021f0       GS_ExceptionPointers       00000001800071f0     MSVCRT:gs_report.obj
 0002:00002898       $unwind$fprintf            0000000180007898     libpopframe009.obj
 0002:000028a4       $unwind$printf             00000001800078a4     libpopframe009.obj
 0002:000028b0       $unwind$?NewObject@JNIEnv_@@QEAAPEAV_jobject@@PEAV_jclass@@PEAU_jmethodID@@ZZ 00000001800078b0     libpopframe009.obj
 0002:000028b0       $unwind$nsk_lcomplain      00000001800078b0     libpopframe009.obj
 0002:000028b0       $unwind$nsk_ldisplay       00000001800078b0     libpopframe009.obj
 0002:000028b8       $unwind$nsk_lvdisplay      00000001800078b8     libpopframe009.obj
 0002:000028b8       $unwind$_RTC_Initialize    00000001800078b8     MSVCRT:initsect.obj
 0002:000028b8       $unwind$_RTC_Terminate     00000001800078b8     MSVCRT:initsect.obj
 0002:000028b8       $unwind$?__scrt_initialize_thread_safe_statics@@YAHXZ 00000001800078b8     MSVCRT:thread_safe_statics.obj
 0002:000028c4       $unwind$nsk_lvcomplain     00000001800078c4     libpopframe009.obj
 0002:000028dc       $unwind$nsk_ltrace         00000001800078dc     libpopframe009.obj
 0002:000028dc       $unwind$__report_gsfailure 00000001800078dc     MSVCRT:gs_report.obj
 0002:000028e4       $unwind$Java_nsk_jvmti_PopFrame_popframe009_getReady 00000001800078e4     libpopframe009.obj
 0002:000028e4       $unwind$nsk_lvtrace        00000001800078e4     libpopframe009.obj
 0002:000028e4       $unwind$__raise_securityfailure 00000001800078e4     MSVCRT:gs_report.obj
 0002:000028e4       $unwind$__scrt_initialize_crt 00000001800078e4     MSVCRT:utility.obj
 0002:000028e4       $unwind$__scrt_initialize_onexit_tables 00000001800078e4     MSVCRT:utility.obj
 0002:000028e4       $unwind$__scrt_release_startup_lock 00000001800078e4     MSVCRT:utility.obj
 0002:000028e4       $unwind$__scrt_uninitialize_crt 00000001800078e4     MSVCRT:utility.obj
 0002:000028e4       $unwind$_onexit            00000001800078e4     MSVCRT:utility.obj
 0002:000028ec       $unwind$nsk_lverify        00000001800078ec     libpopframe009.obj
 0002:000028fc       $unwind$nsk_vprintf        00000001800078fc     libpopframe009.obj
 0002:0000290c       $unwind$nsk_printf         000000018000790c     libpopframe009.obj
 0002:00002914       $unwind$?nsk_jni_lverify@@YAHHPEAUJNIEnv_@@HQEBDH1ZZ 0000000180007914     libpopframe009.obj
 0002:00002928       $unwind$?nsk_jni_check_exception@@YAHPEAUJNIEnv_@@QEBDH@Z 0000000180007928     libpopframe009.obj
 0002:00002944       $unwind$Java_nsk_jvmti_unit_FollowReferences_FollowRefObjects_resetTags 0000000180007944     libpopframe009.obj
 0002:00002944       $unwind$addRefToVerify     0000000180007944     libpopframe009.obj
 0002:00002944       $unwind$nsk_jvmti_resetAgentData 0000000180007944     libpopframe009.obj
 0002:00002944       $unwind$nsk_jvmti_setFailStatus 0000000180007944     libpopframe009.obj
 0002:00002944       $unwind$__scrt_initialize_default_local_stdio_options 0000000180007944     MSVCRT:default_local_stdio_options.obj
 0002:00002944       $unwind$?dllmain_crt_dispatch@@YAHQEAUHINSTANCE__@@KQEAX@Z 0000000180007944     MSVCRT:dll_dllmain.obj
 0002:00002944       $unwind$DllMain            0000000180007944     MSVCRT:dll_dllmain_stub.obj
 0002:00002944       $unwind$__GSHandlerCheck   0000000180007944     MSVCRT:gshandler.obj
 0002:00002944       $unwind$?__scrt_uninitialize_thread_safe_statics@@YAXXZ 0000000180007944     MSVCRT:thread_safe_statics.obj
 0002:00002944       $unwind$__scrt_acquire_startup_lock 0000000180007944     MSVCRT:utility.obj
 0002:00002944       $unwind$__scrt_dllmain_after_initialize_c 0000000180007944     MSVCRT:utility.obj
 0002:00002944       $unwind$__scrt_dllmain_before_initialize_c 0000000180007944     MSVCRT:utility.obj
 0002:00002944       $unwind$__scrt_dllmain_crt_thread_attach 0000000180007944     MSVCRT:utility.obj
 0002:00002944       $unwind$__scrt_dllmain_crt_thread_detach 0000000180007944     MSVCRT:utility.obj
 0002:00002944       $unwind$__scrt_dllmain_uninitialize_c 0000000180007944     MSVCRT:utility.obj
 0002:00002944       $unwind$__scrt_dllmain_uninitialize_critical 0000000180007944     MSVCRT:utility.obj
 0002:00002944       $unwind$atexit             0000000180007944     MSVCRT:utility.obj
 0002:0000294c       $unwind$nsk_jvmti_lverify  000000018000794c     libpopframe009.obj
 0002:00002960       $unwind$exitOnError        0000000180007960     libpopframe009.obj
 0002:00002970       $unwind$Java_nsk_share_jvmti_ArgumentHandler_getAgentOptionsString 0000000180007970     libpopframe009.obj
 0002:00002984       $unwind$Java_nsk_jvmti_unit_FollowReferences_FollowRefObjects_getTag 0000000180007984     libpopframe009.obj
 0002:00002984       $unwind$Java_nsk_share_jvmti_DebugeeClass_checkStatus 0000000180007984     libpopframe009.obj
 0002:00002984       $unwind$agentThreadWrapper 0000000180007984     libpopframe009.obj
 0002:00002994       $unwind$startAgentThreadWrapper 0000000180007994     libpopframe009.obj
 0002:000029b0       $unwind$syncDebuggeeStatus 00000001800079b0     libpopframe009.obj
 0002:000029b0       $unwind$__scrt_dllmain_exception_filter 00000001800079b0     MSVCRT:utility.obj
 0002:000029c4       $unwind$Java_nsk_share_jvmti_DebugeeClass_resetAgentData 00000001800079c4     libpopframe009.obj
 0002:000029cc       $unwind$MA_checkStatus     00000001800079cc     libpopframe009.obj
 0002:000029e0       $unwind$Java_nsk_jvmti_unit_FollowReferences_FollowRefObjects_setTag 00000001800079e0     libpopframe009.obj
 0002:000029f8       $unwind$Java_nsk_jvmti_unit_FollowReferences_FollowRefObjects_addRefToVerify 00000001800079f8     libpopframe009.obj
 0002:00002a14       $unwind$Agent_Initialize   0000000180007a14     libpopframe009.obj
 0002:00002a20       $unwind$Breakpoint         0000000180007a20     libpopframe009.obj
 0002:00002a2c       $unwind$SingleStep         0000000180007a2c     libpopframe009.obj
 0002:00002a2c       $unwind$popFrames          0000000180007a2c     libpopframe009.obj
 0002:00002a2c       $unwind$_DllMainCRTStartup 0000000180007a2c     MSVCRT:dll_dllmain.obj
 0002:00002a3c       $unwind$Java_nsk_jvmti_PopFrame_popframe009_check 0000000180007a3c     libpopframe009.obj
 0002:00002a54       $unwind$capture_previous_context 0000000180007a54     MSVCRT:gs_report.obj
 0002:00002a60       $unwind$__GSHandlerCheckCommon 0000000180007a60     MSVCRT:gshandler.obj
 0002:00002a68       $xdatasym                  0000000180007a68     MSVCRT:amdsecgs.obj
 0002:00002a6c       $unwind$?dllmain_crt_process_attach@@YAHQEAUHINSTANCE__@@QEAX@Z 0000000180007a6c     MSVCRT:dll_dllmain.obj
 0002:00002aa8       $unwind$?fin$0@?0??dllmain_crt_process_attach@@YAHQEAUHINSTANCE__@@QEAX@Z@4HA 0000000180007aa8     MSVCRT:dll_dllmain.obj
 0002:00002aa8       $unwind$?fin$0@?0??dllmain_crt_process_detach@@YAH_N@Z@4HA 0000000180007aa8     MSVCRT:dll_dllmain.obj
 0002:00002aa8       $unwind$?fin$1@?0??dllmain_crt_process_detach@@YAH_N@Z@4HA 0000000180007aa8     MSVCRT:dll_dllmain.obj
 0002:00002ab0       $unwind$?dllmain_crt_process_detach@@YAH_N@Z 0000000180007ab0     MSVCRT:dll_dllmain.obj
 0002:00002b04       $unwind$?dllmain_dispatch@@YAHQEAUHINSTANCE__@@KQEAX@Z 0000000180007b04     MSVCRT:dll_dllmain.obj
 0002:00002b2c       $unwind$?filt$0@?0??dllmain_dispatch@@YAHQEAUHINSTANCE__@@KQEAX@Z@4HA 0000000180007b2c     MSVCRT:dll_dllmain.obj
 0002:00002b34       $unwind$__scrt_is_nonwritable_in_current_image 0000000180007b34     MSVCRT:utility.obj
 0002:00002b54       $unwind$__scrt_is_nonwritable_in_current_image$filt$0 0000000180007b54     MSVCRT:utility.obj
 0002:00002b5c       $unwind$__scrt_fastfail    0000000180007b5c     MSVCRT:utility_desktop.obj
 0002:00002b6c       $unwind$__security_init_cookie 0000000180007b6c     MSVCRT:gs_support.obj
 0002:00002b78       $unwind$__isa_available_init 0000000180007b78     MSVCRT:cpu_disp.obj
 0002:00002b88       $xdatasym                  0000000180007b88     MSVCRT:guard_dispatch.obj
 0002:00002b90       $xdatasym                  0000000180007b90     MSVCRT:guard_xfg_dispatch.obj
 0002:00002ba0       .edata                     0000000180007ba0     popframe009.exp
 0002:00002bc8       rgpv                       0000000180007bc8     popframe009.exp
 0002:00002c08       rgszName                   0000000180007c08     popframe009.exp
 0002:00002c48       rgwOrd                     0000000180007c48     popframe009.exp
 0002:00002c68       szName                     0000000180007c68     popframe009.exp
 0002:00002c78       $N00001                    0000000180007c78     popframe009.exp
 0002:00002c87       $N00002                    0000000180007c87     popframe009.exp
 0002:00002c94       $N00003                    0000000180007c94     popframe009.exp
 0002:00002cbe       $N00004                    0000000180007cbe     popframe009.exp
 0002:00002ceb       $N00005                    0000000180007ceb     popframe009.exp
 0002:00002d30       $N00006                    0000000180007d30     popframe009.exp
 0002:00002d6d       $N00007                    0000000180007d6d     popframe009.exp
 0002:00002db5       $N00008                    0000000180007db5     popframe009.exp
 0002:00002df5       $N00009                    0000000180007df5     popframe009.exp
 0002:00002e32       $N00010                    0000000180007e32     popframe009.exp
 0002:00002e6d       $N00011                    0000000180007e6d     popframe009.exp
 0002:00002e9b       $N00012                    0000000180007e9b     popframe009.exp
 0002:00002ecc       $N00013                    0000000180007ecc     popframe009.exp
 0002:00002efb       $N00014                    0000000180007efb     popframe009.exp
 0002:00002f2a       $N00015                    0000000180007f2a     popframe009.exp
 0002:00002f5f       $N00016                    0000000180007f5f     popframe009.exp
 0002:0000336a       .idata$6                   000000018000836a     kernel32:KERNEL32.dll
 0002:000033ce       .idata$6                   00000001800083ce     vcruntime:VCRUNTIME140.dll
 0002:0000353a       .idata$6                   000000018000853a     ucrt:api-ms-win-crt-runtime-l1-1-0.dll
 0002:0000355c       .idata$6                   000000018000855c     ucrt:api-ms-win-crt-stdio-l1-1-0.dll
 0002:0000357c       .idata$6                   000000018000857c     ucrt:api-ms-win-crt-string-l1-1-0.dll
 0003:00000000       ?codeAttributeName@@3PEBDEB 0000000180009000     libpopframe009.obj
 0003:00000008       ?lineNumberAttributeName@@3PEBDEB 0000000180009008     libpopframe009.obj
 0003:00000010       ?localVarAttributeName@@3PEBDEB 0000000180009010     libpopframe009.obj
 0003:00000018       ?localVarTypeAttributeName@@3PEBDEB 0000000180009018     libpopframe009.obj
 0003:00000020       ?stackMapAttributeName@@3PEBDEB 0000000180009020     libpopframe009.obj
 0003:00000028       ?callBytes@@3PAEA          0000000180009028     libpopframe009.obj
 0003:0000002c       ?allocBytes@@3PAEA         000000018000902c     libpopframe009.obj
 0003:0001aad4       redefineAttempted          0000000180023ad4     libpopframe009.obj
 0003:0001aad8       nsk_context                0000000180023ad8     libpopframe009.obj
 0003:0001aae4       redefineSucceed            0000000180023ae4     libpopframe009.obj
 0003:0001aae8       agentFailed                0000000180023ae8     libpopframe009.obj
 0003:0001aaec       currentAgentStatus         0000000180023aec     libpopframe009.obj
 0003:0001aaf0       context                    0000000180023af0     libpopframe009.obj
 0003:0001aba8       agentThread                0000000180023ba8     libpopframe009.obj
 0003:0001abb0       agentThreadProc            0000000180023bb0     libpopframe009.obj
 0003:0001abb8       agentThreadArg             0000000180023bb8     libpopframe009.obj
 0003:0001abc0       agent_data                 0000000180023bc0     libpopframe009.obj
 0003:0001abd0       jvmti_env                  0000000180023bd0     libpopframe009.obj
 0003:0001abd8       jvm                        0000000180023bd8     libpopframe009.obj
 0003:0001abe0       jni_env                    0000000180023be0     libpopframe009.obj
 0003:0001abe8       checkStatus_func           0000000180023be8     libpopframe009.obj
 0003:0001abf0       ?codeAttributeIndex@@3GA   0000000180023bf0     libpopframe009.obj
 0003:0001abf2       printdump                  0000000180023bf2     libpopframe009.obj
 0003:0001abf3       popDone                    0000000180023bf3     libpopframe009.obj
 0003:0001abf4       ?lineNumberAttributeIndex@@3GA 0000000180023bf4     libpopframe009.obj
 0003:0001abf8       ?localVarAttributeIndex@@3GA 0000000180023bf8     libpopframe009.obj
 0003:0001abfc       ?localVarTypeAttributeIndex@@3GA 0000000180023bfc     libpopframe009.obj
 0003:0001ac00       ?stackMapAttributeIndex@@3GA 0000000180023c00     libpopframe009.obj
 0003:0001ac04       ?stackFrameOffset@@3GA     0000000180023c04     libpopframe009.obj
 0003:0001ac08       ?mode@@3HA                 0000000180023c08     libpopframe009.obj
 0003:0001ac0c       ?constantPoolSize@@3GA     0000000180023c0c     libpopframe009.obj
 0003:0001ac10       ?orig@@3PEBEEB             0000000180023c10     libpopframe009.obj
 0003:0001ac18       ?gen@@3PEAEEA              0000000180023c18     libpopframe009.obj
 0003:0001ac20       ?inputPos@@3PEAEEA         0000000180023c20     libpopframe009.obj
 0003:0001ac28       ?endPos@@3PEBEEB           0000000180023c28     libpopframe009.obj
 0003:0001ac30       ?genPos@@3PEAEEA           0000000180023c30     libpopframe009.obj
 0003:0001ac38       ?markPos@@3PEAEEA          0000000180023c38     libpopframe009.obj
 0003:0001ac40       ?constantPool@@3PEAPEADEA  0000000180023c40     libpopframe009.obj
 0003:0001ac48       ?constantPoolCount@@3GA    0000000180023c48     libpopframe009.obj
 0003:0001ac4c       ?zeroBytes@@3PAEA          0000000180023c4c     libpopframe009.obj
 0003:0001ac50       ?codeLength@@3IA           0000000180023c50     libpopframe009.obj
 0003:0001ac54       result                     0000000180023c54     libpopframe009.obj
 0003:0001ac58       ?map@@3PEAIEA              0000000180023c58     libpopframe009.obj
 0003:0001ac60       ?widening@@3PEACEA         0000000180023c60     libpopframe009.obj
 0003:0001ac68       jvmti                      0000000180023c68     libpopframe009.obj
 0003:0001ac70       caps                       0000000180023c70     libpopframe009.obj
 0003:0001ac80       callbacks                  0000000180023c80     libpopframe009.obj
 0003:0001adb8       breakpointLock             0000000180023db8     libpopframe009.obj
 0003:0001adc0       popFrameLock               0000000180023dc0     libpopframe009.obj
 0003:0001adc8       suspendLock                0000000180023dc8     libpopframe009.obj
 0003:0001add0       midCheckPoint              0000000180023dd0     libpopframe009.obj
 0003:0001add8       midRun                     0000000180023dd8     libpopframe009.obj
 0003:0001ade0       bpCount                    0000000180023de0     libpopframe009.obj
 0003:0001ade4       framesCount                0000000180023de4     libpopframe009.obj
 0003:0001adf0       GS_ExceptionRecord         0000000180023df0     MSVCRT:gs_report.obj
 0003:0001ae90       GS_ContextRecord           0000000180023e90     MSVCRT:gs_report.obj
 0003:0001b360       ?g_tss_cv@@3U_RTL_CONDITION_VARIABLE@@A 0000000180024360     MSVCRT:thread_safe_statics.obj
 0003:0001b368       ?g_tss_event@@3PEAXEA      0000000180024368     MSVCRT:thread_safe_statics.obj
 0003:0001b370       ?g_tss_mutex@@3U_RTL_CRITICAL_SECTION@@A 0000000180024370     MSVCRT:thread_safe_statics.obj
 0003:0001b398       ?g_sleep_condition_variable_cs@@3P6AHPEAU_RTL_CONDITION_VARIABLE@@PEAU_RTL_CRITICAL_SECTION@@K@ZEA 0000000180024398     MSVCRT:thread_safe_statics.obj
 0003:0001b3a0       ?g_wake_all_condition_variable@@3P6AXPEAU_RTL_CONDITION_VARIABLE@@@ZEA 00000001800243a0     MSVCRT:thread_safe_statics.obj
 0003:0001b3ac       ?__proc_attached@@3HA      00000001800243ac     MSVCRT:dll_dllmain.obj
 0003:0001b3c0       ?is_initialized_as_dll@@3_NA 00000001800243c0     MSVCRT:utility.obj
 0003:0001b3c1       ?module_local_atexit_table_initialized@@3_NA 00000001800243c1     MSVCRT:utility.obj
 0003:0001b3c8       ?module_local_atexit_table@@3U_onexit_table_t@@A 00000001800243c8     MSVCRT:utility.obj
 0003:0001b3e0       ?module_local_at_quick_exit_table@@3U_onexit_table_t@@A 00000001800243e0     MSVCRT:utility.obj
